:100000000C945E070C947B070C947B070C947B0785
:100010000C947B070C947B070C947B070C947B0758
:100020000C947B070C947B070C947B070C947B0748
:100030000C947B070C947B070C947B070C947B0738
:100040000C947B070C947B070C947B070C947B0728
:100050000C947B070C94B20C0C947B070C947B07DC
:100060000C947B070C947B07808183848687898A24
:100070008C8E8F9192949597989A9B9D9EA0A2A307
:10008000A5A6A7A9AAACADAFB0B2B3B5B6B7B9BA79
:10009000BCBDBEC0C1C2C4C5C6C8C9CACBCDCECF07
:1000A000D0D2D3D4D5D6D7D9DADBDCDDDEDFE0E1C0
:1000B000E2E3E4E5E6E7E8E9EAEAEBECEDEEEEEFB1
:1000C000F0F1F1F2F3F3F4F5F5F6F6F7F8F8F9F9E3
:1000D000FAFAFAFBFBFCFCFCFDFDFDFDFEFEFEFE5C
:1000E000FEFFFFFFFFFFFFFF0000891112239B327D
:1000F0002446AD573665BF74488CC19D5AAFD3BEF8
:100100006CCAE5DB7EE9F7F88110080193331A2207
:10011000A5562C47B7753E64C99C408DDBBF52AED7
:10012000EDDA64CBFFF976E802218B3010029913E7
:100130002667AF763444BD554AADC3BC588ED19FB7
:100140006EEBE7FA7CC8F5D983310A2091121803C7
:10015000A7772E66B5543C45CBBD42ACD99E508F97
:10016000EFFB66EAFDD874C904428D5316619F7097
:100170002004A9153227BB364CCEC5DF5EEDD7FC77
:100180006888E1997AABF3BA85520C4397711E6087
:10019000A1142805B3373A26CDDE44CFDFFD56EC57
:1001A000E9986089FBBB72AA06638F7214409D5167
:1001B0002225AB343006B9174EEFC7FE5CCCD5DD37
:1001C0006AA9E3B8788AF19B87730E6295501C4147
:1001D000A3352A24B1163807CFFF46EEDDDC54CD17
:1001E000EBB962A8F99A708B088481951AA793B627
:1001F0002CC2A5D33EE1B7F04008C919522BDB3A17
:10020000644EED5F766DFF7C899400859BB712A6E6
:10021000ADD224C3BFF136E0C1184809D33B5A2AF6
:10022000E55E6C4FF77D7E6C0AA583B418869197C6
:100230002EE3A7F23CC0B5D14229CB38500AD91BD6
:10024000666FEF7E744CFD5D8BB502A499961087A6
:10025000AFF326E2BDD034C1C3394A28D11A580BB6
:10026000E77F6E6EF55C7C4D0CC685D71EE597F476
:100270002880A1913AA3B3B2444ACD5B5669DF7896
:10028000600CE91D722FFB3E8DD604C79FF516E466
:10029000A9902081BBB332A2C55A4C4BD7795E6876
:1002A000E11C680DF33F7A2E0EE787F61CC495D546
:1002B0002AA1A3B03882B193466BCF7A5448DD5956
:1002C000622DEB3C700EF91F8FF706E69DD414C526
:1002D000ABB122A0B9923083C77B4E6AD5585C4936
:1002E000E33D6A2CF11E780F2D2D2D2D2D2D2D2D5A
:1002F0002D2D2D2D2D2D2D2D2D2D2D2D2D2D2D2D2E
:100300002D2D2D2D2D2D2D2D2D2D0A004820202079
:100310002020202020205072696E7420636F6E664A
:10032000696775726174696F6E0A0043202020202E
:100330002020202020436C65617220636F6E666907
:100340006775726174696F6E0A004C20202020204E
:10035000202020204C6F616420636F6E6669677592
:10036000726174696F6E0A005320202020202020C3
:1003700020205361766520636F6E666967757261D0
:1003800074696F6E0A00573C5858583E2020202050
:10039000536574207472616E736D697373696F6EE7
:1003A000207461696C2074696D6520696E206D73BD
:1003B0000A00773C5858583E20202020536574206E
:1003C000707265616D626C652074696D6520696E1F
:1003D000206D730A00563C312F303E2020202053E0
:1003E000696C656E74206D6F6465206F6E2F6F662B
:1003F000660A0A00763C312F303E202020205665C8
:1004000072626F7365206D6F6465206F6E2F6F660B
:10041000660A0070693C312F303E202020507269FE
:100420006E7420494E464F206F6E2F6F66660A0A23
:1004300000706D3C312F303E2020205072696E7468
:100440002044415441206F6E2F6F66660A00707021
:100450003C312F303E2020205072696E7420504174
:100460005448206F6E2F6F66660A0070643C312F0F
:10047000303E2020205072696E7420445354206F07
:100480006E2F6F66660A0070733C312F303E20205D
:10049000205072696E7420535243206F6E2F6F6626
:1004A000660A006D613C312F303E2020204175747A
:1004B0006F6D61746963206D657373616765204159
:1004C000434B206F6E2F6F66660A0A006D723C7395
:1004D0007369643E20205265747279206C61737474
:1004E000206D6573736167650A006D733C73736992
:1004F000643E2020536574206D65737361676520C9
:10050000726563697069656E7420535349440A00CB
:100510006D633C63616C6C3E2020536574206D6597
:10052000737361676520726563697069656E7420B5
:1005300063616C6C7369676E0A006C743C732F6145
:100540003E20202053656C6563742073796D626F63
:100550006C207461626C6520287374616E646172D2
:10056000642F616C7465726E617465290A0A006C8F
:10057000733C73796D3E20202053656C6563742055
:1005800073796D626F6C0A006C643C302D393E20CB
:10059000202053657420616E74656E6E61206469FD
:1005A00072656374697669747920696E666F0A0092
:1005B0006C673C302D393E20202053657420616EDD
:1005C00074656E6E61206761696E20696E666F0A80
:1005D000006C683C302D393E20202053657420612A
:1005E0006E74656E6E612068656967687420696EF7
:1005F000666F0A006C703C302D393E202020536518
:100600007420545820706F77657220696E666F0A87
:10061000006C6C6F3C4C4F4E3E2020536574206C38
:100620006174697475646520284E4D45412D666F6F
:10063000726D61742C2065672030373230312E376F
:100640003557290A006C6C613C4C41543E202053C4
:100650006574206C6174697475646520284E4D451D
:10066000412D666F726D61742C20656720343930BE
:10067000332E35304E290A0073323C737369643E61
:10068000202053657420504154483220535349442C
:100690000A0A0073313C737369643E202053657409
:1006A00020504154483120535349440A0073643C5C
:1006B000737369643E2020536574206465737469A4
:1006C0006E6174696F6E20535349440A0073633C32
:1006D000737369643E202053657420796F757220AE
:1006E000535349440A00323C63616C6C3E20202025
:1006F0005365742050415448322063616C6C7369B7
:10070000676E0A0A00313C63616C6C3E2020205306
:1007100065742050415448312063616C6C73696783
:100720006E0A00643C63616C6C3E2020205365744B
:100730002064657374696E6174696F6E2063616CA7
:100740006C7369676E0A00633C63616C6C3E2020C9
:100750002053657420796F75722063616C6C7369C6
:10076000676E0A00233C6D73673E2020202053658E
:100770006E642041505253206D6573736167650A42
:100780000A00403C636D743E2020202053656E6457
:10079000206C6F636174696F6E207570646174653D
:1007A0002028636D74203D206F7074696F6E616CDA
:1007B00020636F6D6D656E74290A00213C6461745D
:1007C000613E20202053656E642072617720706145
:1007D000636B65740A0053657269616C20636F6DA9
:1007E0006D616E64733A0A002D2D2D2D2D2D2D2D4A
:1007F0002D2D2D2D2D2D2D2D2D2D2D2D2D2D2D2D29
:100800002D2D2D2D2D2D2D2D2D2D0A0054582054FC
:1008100061696C3A20256C750A0054582050726545
:10082000616D626C653A20256C750A0053796D62C2
:100830006F6C3A2025630A0053796D626F6C2074E7
:1008400061626C653A207374616E646172640A005F
:1008500053796D626F6C207461626C653A20616CD3
:100860007465726E6174650A0044697265637469C7
:10087000766974793A2025640A004761696E3A20E6
:1008800025640A004865696768743A2025640A008F
:10089000506F7765723A2025640A004175746F2D98
:1008A00061636B206D657373616765733A204F6692
:1008B000660A004175746F2D61636B206D657373FB
:1008C000616765733A204F6E0A0050617468323A6E
:1008D00020252E36732D25640A0050617468313A44
:1008E00020252E36732D25640A0044657374696EC5
:1008F0006174696F6E3A20252E36732D25640A00C7
:1009000043616C6C7369676E3A20252E36732D2512
:10091000640A00436F6E66696775726174696F6E11
:100920003A0A00300A004572726F723A20496E76B8
:10093000616C696420636F6D6D616E640A0045725D
:10094000726F723A20496E76616C69642076616CD0
:10095000756520666F72205458207461696C0A00B6
:100960005458205461696C2073657420746F20257D
:100970006C756D730A004572726F723A20496E761B
:10098000616C69642076616C756520666F72207099
:100990007265616D626C650A00507265616D626CB2
:1009A000652073657420746F20256C756D730A0063
:1009B000310A004D657373616765206175746F2D31
:1009C00061636B2064697361626C65640A00310A5B
:1009D000004D657373616765206175746F2D616388
:1009E0006B20656E61626C65640A00310A005265B5
:1009F0007472696564206C617374206D65737361D2
:100A000067650A00310A000A002D25640A004D6559
:100A1000737361676520726563697069656E743AA6
:100A200020252E367300310A000A002D25640A00A5
:100A30004D65737361676520726563697069656E82
:100A4000743A20252E367300310A0053656C6563B5
:100A5000746564207374616E646172642073796D6F
:100A6000626F6C207461626C650A0053656C65632B
:100A700074656420616C7465726E6174652073794D
:100A80006D626F6C207461626C650A0053796D62EF
:100A90006F6C2073657420746F2025630A004469AD
:100AA0007265637469766974792073657420746FF4
:100AB0002025646465670A00446972656374697619
:100AC0006974792073657420746F206F6D6E690A84
:100AD00000310A00310A004761696E207365742095
:100AE000746F20256464420A00310A00416E746507
:100AF0006E6E612068656967687420736574207420
:100B00006F20256C646D204141540A00310A005069
:100B10006F7765722073657420746F202564770A7F
:100B200000310A004C6F6E677469747564652073D8
:100B3000657420746F20252E39730A00310A004C29
:100B4000617469747564652073657420746F202501
:100B50002E38730A0053696C656E74206D6F64657E
:100B60002064697361626C65640A0053696C656E28
:100B700074206D6F646520656E61626C65640A0047
:100B8000566572626F7365206D6F6465206469736A
:100B900061626C65640A00566572626F7365206DF0
:100BA0006F646520656E61626C65640A00310A00DD
:100BB0005072696E7420494E464F206469736162B9
:100BC0006C65640A00310A005072696E7420494EE7
:100BD000464F20656E61626C65640A00310A005000
:100BE00072696E7420444154412064697361626C7F
:100BF00065640A00310A005072696E7420444154E1
:100C00004120656E61626C65640A00310A005072B1
:100C1000696E7420504154482064697361626C6548
:100C2000640A00310A005072696E742050415448C1
:100C300020656E61626C65640A00310A0050726959
:100C40006E74204453542064697361626C65640A55
:100C500000310A005072696E742044535420656E4E
:100C600061626C65640A00310A005072696E74201A
:100C70005352432064697361626C65640A00310AEF
:100C8000005072696E742053524320656E61626C2D
:100C900065640A00310A0050617468323A20252EDA
:100CA00036732D25640A00310A0050617468313AA8
:100CB00020252E36732D25640A00310A0044657301
:100CC00074696E6174696F6E3A20252E36732D2516
:100CD000640A00310A0043616C6C7369676E3A20E4
:100CE000252E36732D25640A00310A005061746880
:100CF000323A20252E36732D25640A00310A005021
:100D0000617468313A20252E36732D25640A00312E
:100D10000A0044657374696E6174696F6E3A2025C8
:100D20002E36732D25640A00310A0043616C6C7302
:100D300069676E3A20252E36732D25640A00310A24
:100D4000004D6573736167652073656E740A0031C9
:100D50000A004C6F636174696F6E20757064617412
:100D6000652073656E740A00310A005061636B651B
:100D7000742073656E740A000D0A00444154413AB0
:100D800020005B252E36732D25645D2000504154D4
:100D9000483A20005B252E36732D25645D200044E3
:100DA00053543A20005B252E36732D25645D2000B8
:100DB0005352433A2000310A00436F6E66696775EB
:100DC000726174696F6E2073617665640A00300A1F
:100DD000004572726F723A204E6F2073746F7265A5
:100DE0006420636F6E66696775726174696F6E20E7
:100DF000746F206C6F6164210A00436F6E666967CF
:100E000075726174696F6E206C6F616465640A004D
:100E1000310A00436F6E66696775726174696F6E3F
:100E200020636C65617265642E2052657374617213
:100E30007420746F206C6F61642064656661756CEA
:100E400074732E0A002D2D2D2D2D2D2D2D2D2D2D94
:100E50002D2D2D2D0A004D6F64656D207265616426
:100E6000790A0044656661756C7420636F6E66690B
:100E70006775726174696F6E206C6F61646564215F
:100E80000A00756E7369676E65642E696F2F6D69F0
:100E900063726F617072730A004D6963726F4150C3
:100EA00052532076312E30620A002D2D2D2D2D2DFE
:100EB0002D2D2D2D2D2D2D2D2D0A000011241FBE81
:100EC000CFEFD8E0DEBFCDBF11E0A0E0B1E0E0ECB5
:100ED000FDE402C005900D92A234B107D9F716E0E7
:100EE000A2E4B1E001C01D92A23CB107E1F70E946B
:100EF000C8200C94DE260C9400000C942F147894D7
:100F000088EE93E00E94EE084DE757E068EE73E04C
:100F100084EC94E00E944C0D86EB94E00E94AC07B8
:100F200086EB94E09093BF068093BE069093BD0637
:100F30008093BC0684EC94E00C94C9129091C0009C
:100F400095FFFCCF8093C60008958091C00087FF75
:100F5000FCCF8091C6000895CF93DF93CDB7DEB765
:100F60002E970FB6F894DEBF0FBECDBFDC019EE01A
:100F7000FD01892F11928A95E9F71092C50087E645
:100F80008093C400E0ECF0E080818D7F808386E078
:100F90008093C20088E18093C1009E012F5F3F4F84
:100FA000F90111929A95E9F783E08C838EE997E035
:100FB0009A87898785EA97E09C878B878EE0F9017D
:100FC00001900D928A95E1F72E960FB6F894DEBF48
:100FD0000FBECDBFDF91CF910895811106C08091E2
:100FE000C000881F8827881F089580E00895809199
:100FF000C00087FF03C08091C60008958FEF089559
:10100000E0911A06F0911B064FB7F894EB58FF4F8A
:1010100024813581868197814FBF28173907E1F0F8
:10102000E0911A06F0911B062FB7F894EB58FF4F8A
:10103000A481B58182819381A817B90719F48081B1
:10104000918104C0A481B581CD01019695838483EB
:101050008C912FBF90E008958FEF9FEF08950F932D
:101060001F93CF93DF93182FC0911A06D0911B06C0
:10107000FE01E959FF4F8081811124C080E490E096
:101080009E8F8D8F1C8E1B8E1A8E01E00083299AF5
:101090002091090130910A0140910B0150910C01FE
:1010A000A0EBB4E00E9451216056704F8F4F9F4FCC
:1010B00020E43FE140E050E00E9470213B8B2A8B0E
:1010C000009393020FB7F894209105013091060127
:1010D0004091070150910801A0EBB4E00E9451211A
:1010E0006056704F8F4F9F4F20E43FE140E050E04B
:1010F0000E9470213D8B2C8B0FBFE0911A06F0915E
:101100001B065FB7F89423A134A1878D90A12817FF
:10111000390739F425A136A181A192A128173907F1
:1011200061F025A136A183A194A1019741E0281780
:10113000390709F040E0842F01C081E05FBF80FDE6
:10114000DCCFE0911A06F0911B064FB7F894A5A1E9
:10115000B6A11C9325A136A181A192A12817390718
:1011600019F4878D90A103C085A196A1019696A33D
:1011700085A34FBFDF91CF911F910F91089581E01B
:1011800080939202089581E08093920210928000F1
:1011900089E18093810081E896E0909387008093B5
:1011A000860080919202882321F080E480937C0065
:1011B00002C010927C003898409880917E00816037
:1011C00080937E0087E080937B008CEE80937A0092
:1011D0008AB1886F8AB9219A229A08950F931F9332
:1011E000CF93DF93CDB7DEB72E970FB6F894DEBF5F
:1011F0000FBECDBF8C018AECD8011D928A95E9F70C
:1012000010931B0600931A0680E490E0F801968F75
:10121000858FC80180599F4FE859FF4F9183808384
:101220009783868395838483C8018C589F4F9383CB
:101230008283C80183589F4FD801AB58BF4F119686
:101240009C938E9317969C938E93169715969C93CA
:101250008E931497C80184549F4F13969C938E933A
:101260001297C8018796D80190969C938E935F97AA
:1012700096969C938E93959794969C938E93939722
:10128000C8018A599F4F92969C938E93919784E0C0
:1012900090E0A681B7811C924681578122813381DB
:1012A0004217530719F42081318104C02681378108
:1012B0002F5F3F4F378326830197009751F70E9496
:1012C000C3082EE0FE013196DF01822F1D928A9520
:1012D000E9F783E08C838FE298E09A87898780E042
:1012E00098E09C878B87D80101900D922A95E1F7B1
:1012F0002E960FB6F894DEBF0FBECDBFDF91CF9113
:101300001F910F9108950F931F93CF93DF938B013C
:10131000E0911A06F0911B0625A136A134A323A360
:10132000EC01080F191FC017D10721F089910E9405
:101330002F08F9CFDF91CF911F910F910895DC0114
:1013400056968C9156978111E9C058968C91589772
:1013500081119FC093962D913C91949795968D9174
:101360009C9196972817390739F454968D919C9142
:101370005597892B09F45CC059968C915997811126
:1013800003C05A961C925A9781E059968C935997AC
:1013900052968D919C915397009789F593962D9134
:1013A0003C91949795968D919C9196972817390723
:1013B00051F454968D919C915597019755969C9315
:1013C0008E93549721C09396ED91FC9194979196AA
:1013D0008D919C919297E817F90729F45F968D916A
:1013E0009C91909706C09396ED91FC919497CF01B4
:1013F000019694969C938E939397808106C0019753
:1014000053969C938E9352978EE757968C9357974B
:1014100057968C9157978B3191F593962D913C91DE
:10142000949795968D919C9196972817390741F43A
:1014300010929302A959BF4F1C92299880E00895F9
:101440009396ED91FC91949791968D919C919297A2
:10145000E817F90729F45F968D919C91909706C043
:101460009396ED91FC919497CF01019694969C935D
:101470008E939397808157968C93579706C08E577B
:10148000823018F459961C92599781E058968C93A3
:10149000589759962C9159975D968D919C915E978E
:1014A0002223A9F05A962C915A97253080F05A960B
:1014B0001C925A978034910519F485E790E002C098
:1014C00080E490E05E969C938E935D9723C058963F
:1014D0003C91589757962C915797232341F05A9651
:1014E0008C915A978F5F5A968C935A970FC05A9641
:1014F0001C925A978034910519F485E790E002C058
:1015000080E490E05E969C938E935D97330F58969F
:101510003C93589788E056968C9356975D96ED913C
:10152000FC915E975B968D919C915C97E80FF91FFB
:101530009F0131705C963C932E935B9756968C91ED
:101540005697815056968C93FF27E038F10530F07E
:101550008FEF90E0AC014E1B5F0BFA01E859FF4F93
:1015600084912F3F310511F008F080950895EF9296
:10157000FF920F931F93CF93DF93FC018C010154D3
:101580001F4FD8014D915C91DC01A354BF4F4D9387
:101590005C93DC01A859BF4F14968D919C911597CF
:1015A00012962D913C9113978217930721F42D9158
:1015B0003C91119707C014968D919C9115979C01B1
:1015C0002F5F3F4F15963C932E931497EC01888123
:1015D0008602C00111249595879595958795E80118
:1015E000998388837F01D3ECED0EF11CE7012881FC
:1015F00039818F010F531F4FE80139832883840FEE
:10160000951F35952795820F931FE701998388834E
:10161000AF014B535F4F21E0181619060CF020E084
:10162000EA018881880F822B888316968D919C9180
:101630001797EC01688316962D913C911797129697
:101640008D919C9113972817390721F48D919C91C6
:10165000119705C016968D919C9117970196179634
:101660009C938E931697DA019C91892F8695869587
:1016700089278370DF01AA53BF4F833039F48C91DF
:10168000803214F48F5F01C081508C938C91885FFD
:101690008C9380340CF45FC18F738C93DF01A9535A
:1016A000BF4F8C91880F97702BEF290F233010F0CC
:1016B000933009F481608C939C91892F86958927BA
:1016C000809581709685990F892B86878E3709F0D2
:1016D0004EC0DF01AB58BF4F14962D913C9115972A
:1016E0008D919C9111972817390759F416962D91D1
:1016F0003C91179712968D919C9113972817390753
:1017000081F016962D913C91179714968D919C918E
:101710001597019741E02817390709F040E0842F19
:1017200001C081E080FDDCC01696CD91DC91179759
:101730008EE7888316962D913C91179712968D917E
:101740009C9113972817390721F48D919C9111973B
:1017500005C016968D919C911797019617969C93AC
:101760008E93169781E0818B2A9A41E0BCC0982F16
:101770009F779F3719F4118A2A98EDC09189992390
:1017800009F4E9C0982F9F739E3309F4E4C080FFE9
:1017900003C080898068808B87858F5F8787908969
:1017A000883008F4A5C0DF01AB58BF4F82E8890F2D
:1017B000823018F09B3109F04BC014962D913C916A
:1017C00015978D919C9111972817390759F4169602
:1017D0002D913C91179712968D919C9113972817F4
:1017E000390781F016962D913C91179714968D919B
:1017F0009C911597019741E02817390709F040E0BF
:10180000842F01C081E080FD1FC01696CD91DC9130
:1018100017978BE1888316962D913C911797129616
:101820008D919C9113972817390721F48D919C91E4
:10183000119705C016968D919C9117970196179652
:101840009C938E93169704C0118A2A9840E001C099
:1018500041E014962D913C9115978D919C91119793
:101860002817390759F416962D913C91179712961F
:101870008D919C9113972817390781F016962D9119
:101880003C91179714968D919C911597019751E073
:101890002817390709F050E0852F01C081E080FD4D
:1018A0001FC080891696CD91DC9117978883169674
:1018B0002D913C91179712968D919C911397281713
:1018C000390721F48D919C91119705C016968D9141
:1018D0009C911797019617969C938E93169703C029
:1018E000118A2A9840E0108A1786442321F033C0D9
:1018F0009695908B30C0DF01A853BF4F8D919C917E
:101900001197816011969C938E93EB58FF4F248121
:101910003581808191812817390739F426813781F3
:10192000828193812817390761F02681378184816C
:101930009581019741E02817390709F040E0842F8D
:1019400001C081E080FF07C08681978195838483F1
:1019500011961C921E92DF91CF911F910F91FF90D3
:10196000EF9008951F920F920FB60F9211242F93AC
:101970003F934F935F936F937F938F939F93AF9317
:10198000BF93EF93FF9380E286BB609178007091E4
:1019900079007695679576956795605880911A06D7
:1019A00090911B060E94B70A80919302882349F008
:1019B00080911A0690911B060E949F09807F886083
:1019C00001C080E88BB98091B2049091B304A091DA
:1019D000B404B091B5040196A11DB11D8093B20469
:1019E0009093B304A093B404B093B504FF91EF9126
:1019F000BF91AF919F918F917F916F915F914F9127
:101A00003F912F910F900FBE0F901F901895CF927E
:101A1000DF92EF92FF920F931F93CF93DF931F926A
:101A2000CDB7DEB77C01462F82E8860F9701265B93
:101A30003E4F6901823010F06B3149F4F60160814C
:101A400071818BE190E049830E94BF234981D701D6
:101A5000A05BBE4F2C9111965C911197842F90E062
:101A6000FC01E227EE0FFF1FE851FF4F2591349153
:101A7000052F10E0202731272D933C93F60160813C
:101A800071810F90DF91CF911F910F91FF90EF9097
:101A9000DF90CF900C94BF2326E531E0DC01F90103
:101AA0001D923197E9F7FC01E65BFE4F718360837D
:101AB000FC01EE5AFE4F51834083FC01E05BFE4F78
:101AC0002FEF3FEF31832083FC01E25BFE4F318338
:101AD000208308952F923F924F925F926F927F9250
:101AE0008F929F92AF92BF92CF92DF92EF92FF922E
:101AF0000F931F93CF93DF93CDB7DEB7C555D109B1
:101B00000FB6F894DEBF0FBECDBF8C01865B9E4F33
:101B100064969FAF8EAF649728019BEA491A9EEFA7
:101B2000590A5801ACEAAA1AAEEFBA0A7801B4EB26
:101B3000EB1ABEEFFB0A6496EEADFFAD64978081B1
:101B400091810E9481238F3FFFEF9F0709F424C1F9
:101B5000D2012C912111F1C08E37910509F0E1C01D
:101B6000F70140815181C801825B9E4F62969FAF11
:101B70008EAF62974231510508F4C4C0DC018D91EB
:101B80009C91883B904F09F0BDC0D801FE0138966A
:101B9000CE010E962D912695203209F420E0219356
:101BA000E817F907B9F7F801868186958F708E8757
:101BB000D8011796FE013196CF0106962D912695F4
:101BC000203209F420E02193E817F907B9F7F8016A
:101BD0003D96D8011D968C9186958F708F8329969E
:101BE0008FAC2997912C97E0792E61E070E080818D
:101BF00080FF10C028969FAE289729968FAE299710
:101C0000818190E02B969FAF8EAF2B97039709F0C1
:101C100079C057C0B7E0B91568F322242394312C5A
:101C20002C0E3D1E27E0929E200C311C1124CF016A
:101C3000019666969FAF8EAF669780E090E0292D63
:101C400030E06696AEADBFAD66976D906696BFAF5D
:101C5000AEAF66976694B0E26B1201C0612C610171
:101C6000C80ED91ED6011E966C920196863091053B
:101C700041F737969081729ED001739EB00D11246A
:101C8000CC24C394D12CCC0EDD1EAC0DBD1D892FF0
:101C900086958F7054968C9397FF08C0CB0102C035
:101CA000880F991F2A95E2F7882A09C0DB0102C034
:101CB000AA0FBB1F2A95E2F79D01209582229394DB
:101CC00096CF82812C968FAF2C97803FD9F4339694
:101CD00042505109C8018E1B9F0B480F591F609637
:101CE0005FAF4EAF60972E96FFAFEEAF2E97F80125
:101CF000EE5AFE4F0190F081E02D309719F0CE01A1
:101D00000196099581E0D5018C938FEF9FEF629644
:101D1000EEADFFAD629791838083D7011D921C9237
:101D20000ACF8F37910511F4F50134C08B3191053D
:101D300021F481E0D2018C93FECEF5012081222393
:101D400041F1D7012D913C912A34B1E03B0700F5D8
:101D5000A9014F5F5F4FF70151834083F801E20F04
:101D6000F31F8083D801A25BBE4F2D913C91119748
:101D7000F901E827FF27EE0FFF1FE851FF4F85917C
:101D80009491232F3327822793278D939C9301C00F
:101D90001082F2011082CFCECB5ADF4F0FB6F894EB
:101DA000DEBF0FBECDBFDF91CF911F910F91FF908E
:101DB000EF90DF90CF90BF90AF909F908F907F90EB
:101DC0006F905F904F903F902F9008958F929F92C9
:101DD000AF92BF92CF92DF92EF92FF920F931F9339
:101DE000CF93DF938C014B016A017C0180EBE81AF1
:101DF0008EEFF80A8FEF9FEFF701918380835801F0
:101E0000F6EBAF1AFEEFBF0AF501608171818EE734
:101E100090E00E94BF23E401C80CD91CCC15DD055D
:101E200029F06991C8010E94070DF8CFF701608180
:101E3000C1816095C8010E94070D6C2F6095C80193
:101E40000E94070DF501608171818EE790E0DF91BE
:101E5000CF911F910F91FF90EF90DF90CF90BF90A7
:101E6000AF909F908F900C94BF232F923F924F92F0
:101E70005F926F927F928F929F92AF92BF92CF921A
:101E8000DF92EF92FF920F931F93CF93DF93CDB723
:101E9000DEB729970FB6F894DEBF0FBECDBF998786
:101EA00088876B014A012C833D835C0180EBA81A73
:101EB0008EEFB80A8FEF9FEFF5019183808328841E
:101EC0003984F6EB2F1AFEEF3F0AF1016081718130
:101ED0008EE790E00E94BF237601C12CD12CC40173
:101EE00001979B838A83C814D90409F458C091E0F0
:101EF0009983EA81FB81CE16DF0609F01982F7018A
:101F000001900020E9F7CF0101973C016E187F088E
:101F100097E06916710418F026E0622E712C930187
:101F20002E0D3F1D27014216530689F0F2018191C3
:101F30002F0190E02E833F830E946823682F660F55
:101F4000888599850E94070D3F812E81ECCFF6E0B0
:101F50006F16710499F0412C512C86E090E086199F
:101F600097093C014614570448F460E48885998534
:101F70000E94070D9FEF491A590AF4CF89818066A4
:101F8000F7016681660F682B888599850E94070D89
:101F9000FFEFCF1ADF0A87E0E80EF11CA4CF63E061
:101FA000888599850E94070D60EF888599850E9434
:101FB000070DEC80FD800E0D1F1DE016F10641F0AF
:101FC000F70161917F01888599850E94070DF5CF02
:101FD000F501608111816095888599850E94070DC2
:101FE000612F6095888599850E94070DF1016081B8
:101FF00071818EE790E029960FB6F894DEBF0FBE90
:10200000CDBFDF91CF911F910F91FF90EF90DF90A7
:10201000CF90BF90AF909F908F907F906F905F9088
:102020004F903F902F900C94BF2390931E06809367
:102030001D065093B7044093B60470932006609336
:102040001F060895EF92FF920F931F93CF93DF9394
:10205000EC016091B6047091B70480EC90E00E94AE
:10206000BF236091B6047091B70480E090E00E94B5
:10207000BF238E017E0184EBE81A8EEFF80AF70188
:102080008081918102976091B6047091B7049801A4
:102090002C1B3D0B2817390708F5F80181918F019A
:1020A000803C59F48BED90E00E94BF236091B60410
:1020B0007091B7048CED90E00EC08B3D59F48BED20
:1020C00090E00E94BF236091B6047091B7048DED3B
:1020D00090E001C090E00E94BF23D1CF80EC90E05F
:1020E000DF91CF911F910F91FF90EF900C94BF2340
:1020F0008F929F92AF92BF92CF92DF92EF92FF9218
:102100000F931F93CF93DF93EC017B016A01E09162
:102110001F06F09120068189811144C00E943A2354
:1021200090910001891788F4A601B701CE01DF91D3
:10213000CF911F910F91FF90EF90DF90CF90BF90C4
:10214000AF909F908F900C94E60E8FB7F89480908C
:10215000B2049090B304A090B404B090B5048FBFC3
:10216000209101013091020140910301509104013D
:10217000AAE0B0E00E9451214FB7F8940091B20458
:102180001091B3042091B4043091B5044FBF0819E5
:1021900019092A093B0906171707280739070CF000
:1021A000B6CFEACFE0911F06F091200681898823FF
:1021B00009F4ADCF80911D0690911E060E946A0D14
:1021C000E0911F06F0912006E853FF4F8081918136
:1021D000892B41F311821082DF91CF911F910F91D2
:1021E000FF90EF90DF90CF90BF90AF909F908F9037
:1021F0000895282F809121068823A1F0203C01F525
:1022000080910D01811111C010922106409122068A
:102210005091230664E972E080911D0690911E069C
:102220000C947810203C09F079C081E0809321065D
:102230008EEF80930D0110922306109222060895CE
:1022400080912206909123068A3431E0930708F0AA
:1022500065C030910D01009731F43E3F21F42F709D
:1022600020930D01089531111FC02B3D21F481E011
:1022700080931C06089530911C06332349F02C3DB1
:1022800021F02D3D19F42BED01C020EC10921C061D
:10229000AC014F5F5F4F5093230640932206FC0131
:1022A000EC56FD4F20830895313071F430E0AAE000
:1022B000B0E00E943B216093090170930A01809372
:1022C0000B0190930C010895343089F43AE0239F78
:1022D000C0011124AA2797FDA095BA2F809305016C
:1022E00090930601A0930701B0930801089533303D
:1022F00089F43AE0239FC0011124AA2797FDA095F5
:10230000BA2F8093010190930201A0930301B0932F
:1023100004010895323011F42093000108956FEF05
:102320008EE290E00E94132680913201882341F0D2
:1023300083E19EE09F938F930E94F1230F900F9073
:102340008091320181110CC08091E703811108C096
:1023500080E19EE09F938F930E94F1230F900F9056
:102360000895CF938EE290E00E94F525893609F01A
:10237000E3C046E050E068E270E08CE291E00E9449
:10238000E52546E050E062E270E086E291E00E94DE
:10239000E52546E050E06CE170E080E291E00E94CB
:1023A000E52546E050E066E170E088E191E00E94BA
:1023B000E52585E190E00E94F52590E09093E40307
:1023C0008093E30384E190E00E94F52590E09093F0
:1023D000E2038093E10383E190E00E94F52590E021
:1023E00090931F0180931E0182E190E00E94F525E9
:1023F00090E0909317018093160181E190E00E9494
:10240000F52591E0811101C090E09093370180E1C2
:1024100090E00E94F52591E0811101C090E0909339
:1024200036018FE090E00E94F52591E0811101C016
:1024300090E0909335018EE090E00E94F52591E0C8
:10244000811101C090E0909334018DE090E00E94F2
:10245000F52591E0811101C090E0909333018CE06B
:1024600090E00E94F525C1E0811101C0C0E0C09359
:1024700032018BE090E00E94F52591E0811101C0CE
:1024800090E09093E7038AE090E00E94F525809326
:10249000130189E090E00E94F5258093120188E005
:1024A00090E00E94F5258093110187E090E00E9462
:1024B000F5258093100186E090E00E94F525809339
:1024C000150185E090E00E94F5258093140184E0D9
:1024D00090E00E94F52591E0811101C090E0909379
:1024E000DE0382E090E00E94FD25A0E0B0E0809352
:1024F000090190930A01A0930B01B0930C0180E0B5
:1025000090E00E94FD25A0E0B0E08093050190934B
:102510000601A0930701B0930801CC23C1F180917B
:10252000E6038823A1F18AEF9DE09F938F930E9499
:10253000F1230F900F902BC08091E603882381F048
:102540008091E70381110CC080913201882341F012
:1025500081ED9DE09F938F930E94F1230F900F9048
:102560008091E603882381F08091E70381110CC0FC
:1025700080913201811108C08EEC9DE09F938F9372
:102580000E94F1230F900F9081E08093E503CF919B
:10259000089590931E0680931D060E94B11181E05C
:1025A0008093E603809132018823A1F18AEA9EE0BC
:1025B0009F938F930E94F12389E99EE09F938F93CD
:1025C0000E94F12382E89EE09F938F930E94F12363
:1025D0000F900F900F900F900F900F908091E50348
:1025E000882341F083E69EE09F938F930E94F1231E
:1025F0000F900F9086E59EE09F938F930E94F123AA
:1026000085E49EE09F938F930E94F1230F900F909B
:102610000F900F90089546E050E068E270E08CE281
:1026200091E00E94032646E050E062E270E086E21C
:1026300091E00E94032646E050E06CE170E080E209
:1026400091E00E94032646E050E066E170E088E1F8
:1026500091E00E9403266091E30385E190E00E94EF
:1026600013266091E10384E190E00E9413266091BB
:102670001E0183E190E00E9413266091160182E121
:1026800090E00E9413266091370181E190E00E9462
:1026900013266091360180E190E00E94132660913C
:1026A00035018FE090E00E941326609134018EE0A6
:1026B00090E00E941326609133018DE090E00E942B
:1026C0001326609132018CE090E00E941326609105
:1026D000E7038BE090E00E941326609113018AE0EB
:1026E00090E00E9413266091120189E090E00E9420
:1026F00013266091110188E090E00E9413266091FA
:10270000100187E090E00E9413266091150186E099
:1027100090E00E9413266091140185E090E00E94F1
:1027200013266091DE0384E090E00E9413266091FE
:10273000090170910A0182E090E00E9425266091D3
:1027400005017091060180E090E00E94252669E66F
:102750008EE290E00E94132680913201882341F09E
:1027600089EB9DE09F938F930E94F1230F900F9030
:102770008091320181110CC08091E703811108C062
:1027800086EB9DE09F938F930E94F1230F900F9013
:1027900008950F931F939C01CA0146E0E6E2F1E021
:1027A000A2E4B6E001900D924A95E1F74091E10371
:1027B0004093480646E0ECE2F1E0A1EAB6E0019081
:1027C0000D924A95E1F74091E3034093A70646E056
:1027D000E0E2F1E0A9E4B6E001900D924A95E1F75C
:1027E00040911E0140934F0646E0E8E1F1E0A1EB85
:1027F000B6E001900D924A95E1F7409116014093A1
:10280000B70647E0E2E4F6E0A4E2B6E001900D92FC
:102810004A95E1F747E0E1EAF6E0ABE2B6E0019085
:102820000D924A95E1F747E0E9E4F6E0A2E3B6E06D
:1028300001900D924A95E1F747E0E1EBF6E0A9E35C
:10284000B6E001900D924A95E1F78B0144E050E02B
:1028500064E276E00E94350F1F910F9108958F92E8
:102860009F92AF92BF92CF92DF92EF92FF920F931F
:102870001F93CF93DF9300D000D000D0CDB7DEB749
:102880006C01809137018823F9F08091330188230E
:1028900041F080EB9DE09F938F930E94F1230F9076
:1028A0000F90D60116968C911F928F93DF92CF9244
:1028B00085EA9DE09F938F930E94F1230F900F90E4
:1028C0000F900F900F900F9080913601882301F1A7
:1028D00080913301882341F08FE99DE09F938F938E
:1028E0000E94F1230F900F90F60185851F928F9320
:1028F000C60107969F938F9384E99DE09F938F93E2
:102900000E94F1230F900F900F900F900F900F9057
:1029100080913501811105C080913401811144C03D
:1029200036C080913301882341F08DE89DE09F936C
:102930008F930E94F1230F900F908601025F1F4F2B
:10294000E12CF12C4601F6E48F0E911C82E8A82EB2
:102950008DE0B82EF401808190E0E816F906E4F6E7
:10296000D80116968C911F928F931F930F93BF924D
:10297000AF920E94F123BFEFEB1AFB0A095F1F4FD2
:102980000F900F900F900F900F900F90E3CF88E76C
:102990009DE09F938F930E94F1230F900F90809161
:1029A000DE03811136C02DC1809133019601235B76
:1029B0003F4F7901882389F0D90111968C911197A5
:1029C0008F938C918F938BE79DE09F938F930E94C1
:1029D000F1230F900F900F900F9000E010E0560140
:1029E000BBE4AB0EB11CF701808191810817190778
:1029F00070F66091BE067091BF06D501ED91FC9115
:102A0000E00FF11F808190E00E94BF230F5F1F4FF6
:102A1000EACFF601E35BFF4F0190F081E02DEC304F
:102A2000F10508F4EEC0D601A55BBF4F2D913C9196
:102A30007F01E20EF31E80E090E0A12CB12CAE01EC
:102A40004F5F5F4FD7016E917D016B3769F4DA01FB
:102A5000B701FB011191BF011D938D01041B150BE3
:102A600080179107B0F75C0101968730910551F707
:102A7000A114B10409F4C5C081E090E0A1E0F9011E
:102A8000E80FF91F5081FC01E55DFE4F40815417AE
:102A900019F087E090E0A0E00196873091057CF383
:102AA00040E050E0F901E80FF91F60816D3209F450
:102AB000AC0101968A309105ACF341155105A1F0A6
:102AC000F901E40FF51F82816091E3037091E40343
:102AD000803221F4818190E0C09702C090E0869717
:102AE0008617970709F08DC0AA2309F48AC07501DB
:102AF000FEE0EF0EF11CC7010E94C5218C0180E0B1
:102B000090E020E20196F801E80FF91F2083893058
:102B10009105C1F7B60181E090E0E0E0F0E0DB0173
:102B20004D91BD01442331F09801280F391FD9017F
:102B30004C93319601968730910589F7D601169608
:102B40008C91882369F0E00FF11F9DE291838A3018
:102B500018F4805D828304C091E392838A5D83834D
:102B60008AE3F8018083828781E6838783E684870E
:102B70008BE68587DE0112963E9680E090E0019616
:102B80002D9121938A159B05D4F32FB7F89480914A
:102B9000B2049091B304A091B404B091B5042FBFD6
:102BA0002FB7F8944091B2045091B3046091B404EB
:102BB0007091B5042FBF481B590B6A0B7B0B4C352A
:102BC00054446105710560F340911D0650911E0645
:102BD000B701C8010E94C913C80126960FB6F89420
:102BE000DEBF0FBECDBFDF91CF911F910F91FF9040
:102BF000EF90DF90CF90BF90AF909F908F900C940C
:102C00005D2226960FB6F894DEBF0FBECDBFDF91D2
:102C1000CF911F910F91FF90EF90DF90CF90BF90D9
:102C2000AF909F908F9008956F927F929F92AF92F6
:102C3000BF92CF92DF92EF92FF920F931F93CF93A9
:102C4000DF931F92CDB7DEB75C018B016A017B0178
:102C500084E1E80EF11C209113012A3098F4809150
:102C600012018A3078F4809111018A3058F48091F1
:102C70001001893038F47B01EBE1EE0EF11C992450
:102C8000939401C0912CC70129830E94C5213C0166
:102C90008DE3F30180838091150181878091140178
:102CA000838B88E0E9E9F6E0D301119601900D925B
:102CB0008A95E1F789E0E8EAF6E0D3011A960190F7
:102CC0000D928A95E1F72981911003C0C3014496C2
:102CD00017C080E5F301848B88E4858B87E4868BBD
:102CE000205D278B80911201805D808F8091110182
:102CF000805D818F80911001805D828FC3014B9632
:102D00000115110521F0A801B5010E947023A6014B
:102D1000B701C3010E94C913C3010F90DF91CF9186
:102D20001F910F91FF90EF90DF90CF90BF90AF90E9
:102D30009F907F906F900C945D228F929F92AF92A4
:102D4000BF92CF92DF92EF92FF920F931F93CF9398
:102D5000DF935C016A018B016434710510F003E4B8
:102D600010E078012FE0E20EF11CC7010E94C5219E
:102D7000EC018AE3888387E090E020E030E001976F
:102D8000009769F0F901E05BF94F40814423B9F302
:102D90002F5F3F4FFE01E20FF31F4083F0CF809182
:102DA0000E0190910F018F3F4FEF940779F0FE01D4
:102DB000E20FF31F4DE241838A3091054CF42E5F00
:102DC0003F4FFE01E20FF31F805D808380E209C068
:102DD00091E392832D5F3F4FFE01E20FF31F8A5D67
:102DE000F4CF293031053CF42F5F3F4FFE01E20F55
:102DF000F31F8083F6CFFE01E20FF31F8AE3818386
:102E00000115110581F0A801B501CE010B960E94B4
:102E10007023A801B50186E596E00E947023109307
:102E20004106009340068091DF039091E0030196F4
:102E3000883E23E092072CF49093E0038093DF0315
:102E400004C01092E0031092DF03FE01E00FF11FB7
:102E50008BE783870091DF031091E0039AE0892ECE
:102E6000912CC801B4010E945C219C0144E6A42E6F
:102E7000B12CC801B5010E945C21821B930BB401E7
:102E80000E945C21AB01C801861B970B821B930B30
:102E9000B5010E945C21605D6487405D4587205DCF
:102EA0002687A601B701CE010E94C913CE01DF918A
:102EB000CF911F910F91FF90EF90DF90CF90BF9037
:102EC000AF909F908F900C945D222091DF03309102
:102ED000E003215031093093E0032093DF03609138
:102EE000400670914106AC0186E596E00C949D1673
:102EF00083E199E09F938F930E94F1238091E403F3
:102F00008F938091E3038F938CE291E09F938F9353
:102F100080E099E09F938F930E94F1238091E203D8
:102F20008F938091E1038F9386E291E09F938F933B
:102F30008AEE98E09F938F930E94F12380911F0166
:102F40008F9380911E018F9380E291E09F938F93E6
:102F50008AED98E09F938F930E94F123809117014F
:102F60008F93809116018F9388E191E09F938F93C7
:102F70008AEC98E09F938F930E94F1238DB79EB7C0
:102F80004A960FB6F8949EBF0FBE8DBF8091DE03A8
:102F9000882319F083EB98E002C08BE998E09F93B7
:102FA0008F930E94F1230F900F90809113018A302C
:102FB00061F01F928F9380E998E09F938F930E9416
:102FC000F1230F900F900F900F90809112018A3093
:102FD00061F01F928F9384E898E09F938F930E94F3
:102FE000F1230F900F900F900F90809111018A3074
:102FF00061F01F928F938AE798E09F938F930E94CE
:10300000F1230F900F900F900F90809110018A3054
:1030100061F01F928F9389E698E09F938F930E94AF
:10302000F1230F900F900F900F90809115018C3528
:1030300041F480E598E09F938F930E94F1230F90D5
:103040000F90809115018F3241F488E398E09F93AF
:103050008F930E94F1230F900F90809114011F9283
:103060008F938CE298E09F938F930E94F12380913D
:103070000C018F9380910B018F9380910A018F93A4
:10308000809109018F938AE198E09F938F930E942A
:10309000F123809108018F93809107018F93809194
:1030A00006018F93809105018F938CE098E09F93A8
:1030B0008F930E94F1238DB79EB740960FB6F89478
:1030C0009EBF0FBE8DBF089588EE97E09F938F93AC
:1030D0000E94F12386ED97E09F938F930E94F12346
:1030E0008BEB97E09F938F930E94F12382E897E008
:1030F0009F938F930E94F12384E697E09F938F9391
:103100000E94F12387E497E09F938F930E94F1231D
:1031100083E297E09F938F930E94F12385E097E0ED
:103120009F938F930E94F12386EE96E09F938F9357
:103130000E94F1238DEC96E09F938F930E94F123E0
:103140008DEA96E09F938F930E94F12383E996E0A6
:103150009F938F930E94F12388E796E09F938F932C
:103160000E94F12385E496E09F938F930E94F123C0
:1031700081E196E09F938F930E94F12384EF95E085
:103180009F938F930E94F1238DB79EB780960FB6C1
:10319000F8949EBF0FBE8DBF81ED95E09F938F93F6
:1031A0000E94F12380EB95E09F938F930E94F1237F
:1031B00088E895E09F938F930E94F1238FE695E036
:1031C0009F938F930E94F1238AE395E09F938F93BF
:1031D0000E94F12380E195E09F938F930E94F12359
:1031E0008AEE94E09F938F930E94F1238CEC94E0FD
:1031F0009F938F930E94F12383EA94E09F938F9390
:103200000E94F12387E894E09F938F930E94F1231B
:103210008BE694E09F938F930E94F1238EE494E0D9
:103220009F938F930E94F12381E394E09F938F9368
:103230000E94F12383E194E09F938F930E94F123F6
:1032400084EF93E09F938F930E94F12385ED93E0A9
:103250009F938F930E94F1238DB79EB780960FB6F0
:10326000F8949EBF0FBE8DBF82EB93E09F938F9328
:103270000E94F12386E893E09F938F930E94F123AD
:1032800088E693E09F938F930E94F1238AE493E072
:103290009F938F930E94F1238BE293E09F938F93F0
:1032A0000E94F1238CE093E09F938F930E94F1237F
:1032B00088EE92E09F938F930E94F1238DB79EB783
:1032C0000E960FB6F8949EBF0FBE8DBF0895EF9275
:1032D000FF920F931F93CF93DF9300D000D0CDB711
:1032E000DEB78C016115710509F447C7FC018081C7
:1032F000813209F56230710508F4FAC6615071092E
:10330000C80101960E94C91380913201882341F0BF
:103310008BE69DE09F938F930E94F1230F900F9077
:1033200080913201811129C78091E703811125C75E
:1033300088E69DE0F3C68034E9F461507109C80164
:1033400001960E94141680913201882341F082E593
:103350009DE09F938F930E94F1230F900F90809197
:10336000320181110AC78091E703811106C78FE4FA
:103370009DE0D4C68332E9F461507109C801019619
:103380000E949D1680913201882341F081E49DE0E6
:103390009F938F930E94F1230F900F9080913201A1
:1033A0008111EBC68091E7038111E7C68EE39DE0B2
:1033B000B5C6883619F40E946418DFC6883419F43B
:1033C0000E947817DAC6833519F40E940B13D5C60C
:1033D000833419F40E948F11D0C68C3419F40E94E2
:1033E000B111CBC6833609F052C06430710508F4C0
:1033F0007FC6ECE2F1E081E090E09C0121503109D0
:1034000086179707A9F08730910581F0D801A80F9A
:10341000B91F2C91222331F02A3021F02D3011F0E8
:10342000208301C0108201963196E7CF26E030E07C
:103430002630310539F0F901E45DFE4F10822F5F2F
:103440003F4FF6CF809132018823B1F08091E403A1
:103450008F938091E3038F938CE291E09F938F93FE
:103460008BE29DE09F938F930E94F1230F900F902A
:103470000F900F900F900F908091320181117DC6B7
:103480008091E703811179C688E29DE047C68436C2
:1034900009F052C06430710508F42AC6E6E2F1E092
:1034A00081E090E09C012150310986179707A9F02F
:1034B0008730910581F0D801A80FB91F2C912223E4
:1034C00031F02A3021F02D3011F0208301C010821C
:1034D00001963196E7CF26E030E02630310539F00D
:1034E000F901EA5DFE4F10822F5F3F4FF6CF8091CA
:1034F00032018823B1F08091E2038F938091E10340
:103500008F9386E291E09F938F9382E19DE09F935A
:103510008F930E94F1230F900F900F900F900F90B8
:103520000F9080913201811128C68091E7038111AB
:1035300024C68FE09DE0F2C5813309F052C06230AD
:10354000710508F4D5C5E0E2F1E081E090E09C016E
:103550002150310986179707A9F08730910581F02E
:10356000D801A80FB91F2C91222331F02A3021F065
:103570002D3011F0208301C0108201963196E7CFE3
:1035800026E030E02630310539F0F901E05EFE4FEB
:1035900010822F5F3F4FF6CF809132018823B1F028
:1035A00080911F018F9380911E018F9380E291E0A3
:1035B0009F938F938FEF9CE09F938F930E94F123B3
:1035C0000F900F900F900F900F900F9080913201FD
:1035D0008111D3C58091E7038111CFC58CEF9CE0A9
:1035E0009DC5823309F052C06230710508F480C570
:1035F000E8E1F1E081E090E09C012150310986177B
:103600009707A9F08730910581F0D801A80FB91F5D
:103610002C91222331F02A3021F02D3011F020831B
:1036200001C0108201963196E7CF26E030E02630C7
:10363000310539F0F901E85EFE4F10822F5F3F4FF0
:10364000F6CF809132018823B1F0809117018F93DA
:10365000809116018F9388E191E09F938F938CEE78
:103660009CE09F938F930E94F1230F900F900F90F7
:103670000F900F900F908091320181117EC5809143
:10368000E70381117AC589EE9CE048C5833709F0CC
:1036900011C16330710508F42BC57B01F1E0EF1A0D
:1036A000F108F8018181833609F03FC0F2E0EF169E
:1036B000F10449F0F80183819FEC980F993018F4D8
:1036C00090E0869704C0F801828190E0C0979093C3
:1036D000E4038093E303809132018823B1F0809169
:1036E000E4038F938091E3038F938CE291E09F93A7
:1036F0008F9386ED9CE09F938F930E94F1230F9010
:103700000F900F900F900F900F90809132018111C8
:103710000CC08091E703811108C083ED9CE09F936A
:103720008F930E94F1230F900F90F80181818436CE
:1037300009F03FC0F2E0EF16F10449F0F80183818F
:103740009FEC980F993018F490E0869704C0F80128
:10375000828190E0C0979093E2038093E10380918F
:1037600032018823B1F08091E2038F938091E103CD
:103770008F9386E291E09F938F938DEB9CE09F93D4
:103780008F930E94F1230F900F900F900F900F9046
:103790000F908091320181110CC08091E70381115B
:1037A00008C08AEB9CE09F938F930E94F1230F90B7
:1037B0000F90F80181818133F1F583819FEC980F9F
:1037C0009930C8F5F2E0EF16F10419F090E0869711
:1037D00004C0F801828190E0C09790931F0180930C
:1037E0001E01809132018823B1F080911F018F93D7
:1037F00080911E018F9380E291E09F938F938AEADC
:103800009CE09F938F930E94F1230F900F900F9055
:103810000F900F900F908091320181110CC0809118
:10382000E703811108C087EA9CE09F938F930E9471
:10383000F1230F900F90F8018181823309F09DC42C
:1038400083819FEC980F993008F097C4F2E0EF164F
:10385000F10419F090E0869704C0F801828190E0AD
:10386000C0979093170180931601809132018823AD
:10387000B1F0809117018F93809116018F9388E1A9
:1038800091E09F938F9387E99CE09F938F930E9491
:10389000F1230F900F900F900F900F900F90809149
:1038A000320181116AC48091E703811166C484E901
:1038B0009CE034C4803709F031C16330710508F4ED
:1038C00017C4F80181818337C9F592818091320153
:1038D0009133C1F491E090933701882341F081E85E
:1038E0009CE09F938F930E94F1230F900F90809103
:1038F0003201811123C08091E70381111FC08EE73F
:103900009CE016C010923701882341F08AE69CE0C3
:103910009F938F930E94F1230F900F90809132011B
:1039200081110CC08091E703811108C087E69CE0FB
:103930009F938F930E94F1230F900F90F801818144
:103940008436C9F59281809132019133C1F491E0BE
:1039500090933601882341F084E59CE09F938F93F8
:103960000E94F1230F900F9080913201811123C0AA
:103970008091E70381111FC081E59CE016C0109281
:103980003601882341F08DE39CE09F938F930E9442
:10399000F1230F900F908091320181110CC0809122
:1039A000E703811108C08AE39CE09F938F930E94F4
:1039B000F1230F900F90F80181818037C9F5928132
:1039C000809132019133C1F491E0909335018823C5
:1039D00041F086E29CE09F938F930E94F1230F9029
:1039E0000F9080913201811123C08091E7038111F2
:1039F0001FC083E29CE016C010923501882341F07D
:103A00008EE09CE09F938F930E94F1230F900F9084
:103A10008091320181110CC08091E703811108C0AF
:103A20008BE09CE09F938F930E94F1230F900F9067
:103A3000F80181818D36C9F59281809132019133EF
:103A4000C1F491E090933401882341F087EF9BE02B
:103A50009F938F930E94F1230F900F9080913201DA
:103A6000811123C08091E70381111FC084EF9BE087
:103A700016C010923401882341F08FED9BE09F9394
:103A80008F930E94F1230F900F908091320181114A
:103A90000CC08091E703811108C08CED9BE09F93DF
:103AA0008F930E94F1230F900F90F8018181893646
:103AB00009F063C39281809132019133C1F491E0A6
:103AC00090933301882341F088EC9BE09F938F9380
:103AD0000E94F1230F900F908091320181114DC30C
:103AE0008091E703811149C385EC9BE017C31092D5
:103AF0003301882341F080EB9BE09F938F930E94DA
:103B0000F1230F900F9080913201811136C3809183
:103B1000E703811132C38DEA9BE000C3863779F455
:103B2000F8018181813331F481E08093320187E9AA
:103B30009BE0F4C21092320180E89BE0EFC2863530
:103B400089F4F8018181813341F481E08093E703B6
:103B5000109232018BE69BE0E1C21092E70385E50B
:103B60009BE0DCC28C3609F040C16330710508F47B
:103B7000BFC2F80181818C3609F05BC061507109C8
:103B80008281813649F56A30710508F4F6C288E011
:103B90003396A9E9B6E001900D928A95E1F78091FC
:103BA0003201882371F089E996E09F938F938FE328
:103BB0009BE09F938F930E94F1230F900F900F90A3
:103BC0000F90809132018111D8C28091E703811159
:103BD000D4C28CE39BE0A2C28F3609F0CEC26B3018
:103BE000710508F4CAC289E0F8013396A8EAB6E084
:103BF00001900D928A95E1F780913201882371F04E
:103C000088EA96E09F938F9384E29BE09F938F9343
:103C10000E94F1230F900F900F900F90809132012E
:103C20008111ABC28091E7038111A7C281E29BE0C1
:103C300075C2803731F5F801828180538A3008F0EF
:103C40009CC28093130190913201992379F0889F4F
:103C5000C00111249F938F938FE09BE09F938F93DC
:103C60000E94F1230F900F900F900F9080913201DE
:103C7000811183C28091E70381117FC28CE09BE0B8
:103C80004DC28836C1F5F801828180538A3008F030
:103C900074C28093120190913201992309F1A1E03D
:103CA000B0E002C0AA0FBB1F8A95E2F728EE33E00E
:103CB0000E944A2128E431E040E050E00E94922135
:103CC0005F934F933F932F938CEE9AE09F938F9344
:103CD0000E94F1230F900F900F900F900F900F9074
:103CE00080913201811149C28091E703811145C25F
:103CF00089EE9AE013C2873619F5F8018281805364
:103D00008A3008F03AC280931101909132019923D0
:103D100061F01F928F9387ED9AE09F938F930E949B
:103D2000F1230F900F900F900F908091320181112D
:103D300024C28091E703811120C284ED9AE0EEC194
:103D40008436D1F5F801828180538A3008F015C29B
:103D5000893009F488E0809310018091320181114B
:103D60000CC08091E703811108C081ED9AE09F9318
:103D70008F930E94F1230F900F908091320188233E
:103D800009F4FBC180911001811108C088EB9AE011
:103D90009F938F930E94F1230F900F9080911001B9
:103DA000882309F4EAC1FDE28F9FC00111249F938B
:103DB0008F938EE99AE010C0833709F0B6C1F801FD
:103DC00082818093140190913201992309F4D5C125
:103DD0001F928F938CE89AE09F938F930E94F12318
:103DE0000F900F900F900F90C8C18D3609F01BC136
:103DF0006230710508F47CC1CB010197F801218183
:103E0000233609F061C0019709F4B7C1E0E5F6E097
:103E1000D80112966250710980E090E086179707EA
:103E200081F08630910569F02D91222331F02A30FE
:103E300021F02D3011F0208301C0108201963196BF
:103E4000EDCF8630910531F0FC01E05BF94F108237
:103E50000196F7CF80913201882359F180E596E0F1
:103E60009F938F9380E39AE09F938F930E94F12317
:103E700080910E0190910F010F900F900F900F9075
:103E80008F3FFFEF9F0769F09F938F938BE29AE03C
:103E90009F938F930E94F1230F900F900F900F909C
:103EA00008C089E29AE09F938F930E94F1230F90BC
:103EB0000F9080913201811160C18091E7038111DF
:103EC0005CC186E29AE02AC1233709F058C08130EC
:103ED000910509F452C1F801029721F0838190E025
:103EE000869703C0828190E0C09790930F018093E2
:103EF0000E0180910E0190910F01409730F08FEFED
:103F00009FEF90930F0180930E01809132018823DF
:103F100059F180E596E09F938F938EE09AE09F930E
:103F20008F930E94F12380910E0190910F010F90C9
:103F30000F900F900F908F3FFFEF9F0769F09F93B7
:103F40008F9389E09AE09F938F930E94F1230F90C3
:103F50000F900F900F9008C087E09AE09F938F9387
:103F60000E94F1230F900F9080913201811105C1C1
:103F70008091E703811101C184E09AE0CFC022372C
:103F8000D1F4CA010E94651780913201882341F063
:103F90008EEE99E09F938F930E94F1230F900F90E4
:103FA000809132018111E9C08091E7038111E5C060
:103FB0008BEE99E0B3C0213609F0DFC0F8019281A1
:103FC000809132019133C1F491E09093DE03882314
:103FD00041F081ED99E09F938F930E94F1230F9020
:103FE0000F90809132018111C8C08091E703811147
:103FF000C4C08EEC99E092C01092DE03882341F099
:1040000083EB99E09F938F930E94F1230F900F9081
:10401000809132018111B1C08091E7038111ADC05F
:1040200080EB99E07BC0873761F56230710508F459
:104030005FC0AB0141505109B8016F5F7F4FCE01A6
:1040400001960E947023CE0101960E944A2380317E
:10405000F7E29F0798F4AA2797FDA095BA2F8093BF
:10406000090190930A01A0930B01B0930C01BF9337
:10407000AF939F938F9389E999E02CC086E799E0ED
:104080004DC08735A9F56230710590F1AB01415003
:104090005109B8016F5F7F4FCE0101960E947023D6
:1040A000CE0101960E944A23803127E29207E8F46C
:1040B000AA2797FDA095BA2F80930501909306013A
:1040C000A0930701B0930801BF93AF939F938F9381
:1040D00080E699E09F938F930E94F1230F900F90B9
:1040E0000F900F900F900F9048C08EE399E016C08C
:1040F00080913201882341F086E299E09F938F936B
:104100000E94F1230F900F9080913201811135C0F0
:104110008091E703811131C083E299E09F938F93EF
:104120000E94F1230F900F9028C0843731F5F801D9
:10413000928180913201913641F49CE59093150172
:10414000882381F08BE69AE007C09FE290931501E7
:10415000882341F08BE49AE09F938F930E94F12390
:104160000F900F9080913201811107C08091E70379
:10417000811103C088E49AE0D1CF0F900F900F9087
:104180000F90DF91CF911F910F91FF90EF900895C5
:104190000E947F078FB7F894C090B204D090B30408
:1041A000E090B404F090B5048FBFC1E084EC94E0DB
:1041B0000E946A0D8091420181112CC00E94ED077E
:1041C000882341F10E94F707282F30E03093460101
:1041D000209345012091430130914401F901E95BAD
:1041E000FE4FA9014F5F5F4F80835093440140937E
:1041F00043012934314010F0C09342018FB7F89445
:10420000C090B204D090B304E090B404F090B50430
:104210008FBF1BC08091430190914401892BA9F06D
:104220002FB7F8948091B2049091B304A091B40494
:10423000B091B5042FBF8C199D09AE09BF094597F0
:10424000A105B10514F0C093420180914201882379
:1042500009F4ACCF609143017091440144EC54E007
:1042600087E491E00E946719109242011092440184
:10427000109243019BCFA29FB001B39FC001A39FA7
:10428000700D811D1124911DB29F700D811D11248F
:10429000911D08950E943B21B7FF0895821B930B47
:1042A00008950E943B21A59F900DB49F900DA49F5F
:1042B000800D911D1124089597FB072E16F400948C
:1042C00007D077FD09D00E94B12107FC05D03EF44C
:1042D000909581959F4F0895709561957F4F0895B2
:1042E000A1E21A2EAA1BBB1BFD010DC0AA1FBB1FFA
:1042F000EE1FFF1FA217B307E407F50720F0A21B6C
:10430000B30BE40BF50B661F771F881F991F1A94D8
:1043100069F760957095809590959B01AC01BD0102
:10432000CF010895052E97FB1EF400940E94A92149
:1043300057FD07D00E94702107FC03D04EF40C9467
:10434000A92150954095309521953F4F4F4F5F4F94
:10435000089590958095709561957F4F8F4F9F4FF1
:104360000895AA1BBB1B51E107C0AA1FBB1FA617BC
:10437000B70710F0A61BB70B881F991F5A95A9F70E
:1043800080959095BC01CD010895CF93DF93823045
:10439000910510F482E090E0E091BA06F091BB063E
:1043A00020E030E0A0E0B0E0309739F14081518169
:1043B00048175907B8F04817590771F4828193815B
:1043C000109729F013969C938E9312972CC090937C
:1043D000BB068093BA0627C02115310531F042177C
:1043E000530718F0A901DB0101C0EF019A01BD01DB
:1043F000DF010280F381E02DD7CF21153105F9F0DF
:10440000281B390B2430310580F48A819B8161158A
:10441000710521F0FB019383828304C09093BB0656
:104420008093BA06FE01329644C0FE01E20FF31FEC
:104430008193919322503109398328833AC0209186
:10444000B8063091B906232B41F420913A013091FE
:104450003B013093B9062093B80620913801309182
:1044600039012115310541F42DB73EB740913C018A
:1044700050913D01241B350BE091B806F091B9062F
:10448000E217F307A0F42E1B3F0B2817390778F02B
:10449000AC014E5F5F4F2417350748F04E0F5F1F8A
:1044A0005093B9064093B8068193919302C0E0E01F
:1044B000F0E0CF01DF91CF910895CF93DF93009784
:1044C00009F487C0FC01329713821282C091BA06A8
:1044D000D091BB06209781F420813181280F391FAC
:1044E0008091B8069091B9068217930779F5F093F9
:1044F000B906E093B8066DC0DE0120E030E0AE17EB
:10450000BF0750F412964D915C9113979D01411590
:10451000510509F1DA01F3CFB383A28340815181C0
:10452000840F951F8A179B0771F48D919C911197A9
:10453000840F951F02969183808312968D919C9192
:104540001397938382832115310529F4F093BB06D9
:10455000E093BA063EC0D9011396FC93EE931297EE
:104560004D915D91A40FB51FEA17FB0779F4808187
:104570009181840F951F0296D90111969C938E9379
:104580008281938113969C938E931297E0E0F0E0E2
:104590008A819B81009719F0FE01EC01F9CFCE01D1
:1045A000029628813981820F931F2091B80630919D
:1045B000B9062817390769F4309729F41092BB0619
:1045C0001092BA0602C013821282D093B906C09329
:1045D000B806DF91CF9108958F929F92AF92BF92CC
:1045E000CF92DF92EF92FF92CF93DF93EC0168813D
:1045F00079818A819B81611571058105910521F47D
:1046000064E279ED8BE597E02DE133EF41E050E096
:104610000E94922149015A019B01AC01A7EAB1E431
:104620000E9451216B017C01ACEEB4EFA501940115
:104630000E94A226C60ED71EE81EF91EF7FE06C06F
:1046400081E0C81AD108E10880E8F80AC882D98256
:10465000EA82FB82C6019F77DF91CF91FF90EF90B6
:10466000DF90CF90BF90AF909F908F9008950E9461
:10467000EC2208958EE391E00E94EC220895A0E0E0
:10468000B0E080933E0190933F01A0934001B0932E
:1046900041010895FC0188279927E894219120324F
:1046A000E9F3293010F02E30C8F32B3241F02D32CF
:1046B00039F4689404C00E947923820F911D2191DE
:1046C00020532A30C0F31EF4909581959F4F089592
:1046D0009111089581568A5108F4805285580895A1
:1046E000FB01DC0102C001900D9241505040D8F70F
:1046F00008957AE0979F902D879F802D910D11242A
:104700000895CF93DF93EC012B8120FF33C026FF68
:104710000AC02F7B2B838E819F8101969F838E837E
:104720008A8190E029C022FF0FC0E881F981808151
:10473000992787FD9095009719F420622B831AC062
:104740003196F983E8830EC0EA85FB85099597FFCA
:1047500009C02B81019611F480E101C080E2822B17
:104760008B8308C02E813F812F5F3F4F3F832E8375
:10477000992702C08FEF9FEFDF91CF9108950F939C
:104780001F93CF93DF93182F092FEB018B8181FDAE
:1047900003C08FEF9FEF20C082FF10C04E815F816A
:1047A0002C813D81421753077CF4E881F9819F01F8
:1047B0002F5F3F4F39832883108306C0E885F98532
:1047C000812F0995892B29F72E813F812F5F3F4F3C
:1047D0003F832E83812F902FDF91CF911F910F91D7
:1047E0000895A0E0B0E0E7EFF3E20C94B526FE01F7
:1047F0003796619171910EEB16E0D8018D919C91E5
:10480000DC0113962C911397286013962C93AF011B
:104810000E941324D801ED91FC912381277F2383EB
:10482000E4E00C94D126ACE0B0E0E9E1F4E20C94D1
:10483000A7267C016B018A01FC0117821682838105
:1048400081FFBDC1CE0101964C01F7019381F601B4
:1048500093FD859193FF81916F01882309F4ABC18A
:10486000853239F493FD859193FF81916F018532F3
:1048700029F4B70190E00E94BF23E7CF512C312CDF
:1048800020E02032A0F48B3269F030F4803259F00D
:10489000833269F420612CC08D3239F0803339F4D1
:1048A000216026C02260246023C0286021C027FD2B
:1048B00027C030ED380F3A3078F426FF06C0FAE012
:1048C0005F9E300D1124532E13C08AE0389E300DA8
:1048D0001124332E20620CC08E3221F426FD6BC1D0
:1048E000206406C08C3611F4206802C0883641F47A
:1048F000F60193FD859193FF81916F018111C1CFE5
:10490000982F9F7D9554933028F40C5F1F4FFFE341
:10491000F9830DC0833631F0833771F0833509F0A8
:104920005BC022C0F801808189830E5F1F4F442441
:104930004394512C540115C03801F2E06F0E711CE4
:10494000F801A080B18026FF03C0652D70E002C091
:104950006FEF7FEFC5012C870E9436262C01830163
:104960002C852F77222E17C03801F2E06F0E711CB4
:10497000F801A080B18026FF03C0652D70E002C061
:104980006FEF7FEFC5012C870E942B262C012C8511
:104990002068222E830123FC1BC0832D90E0481643
:1049A0005906B0F4B70180E290E00E94BF233A9428
:1049B000F4CFF50127FC859127FE81915F01B701B6
:1049C00090E00E94BF2331103A94F1E04F1A510851
:1049D0004114510471F7E5C0843611F0893639F578
:1049E000F80127FF07C060817181828193810C5F8C
:1049F0001F4F08C060817181882777FD8095982FAF
:104A00000E5F1F4F2F76B22E97FF09C090958095AD
:104A1000709561957F4F8F4F9F4F2068B22E2AE08F
:104A200030E0A4010E944126A82EA81844C0853772
:104A300029F42F7EB22E2AE030E025C0F22FF97F34
:104A4000BF2E8F36C1F018F4883579F0B4C08037A6
:104A500019F0883721F0AFC02F2F2061B22EB4FE9D
:104A60000DC08B2D8460B82E09C024FF0AC09F2F73
:104A70009660B92E06C028E030E005C020E130E0A5
:104A800002C020E132E0F801B7FE07C06081718109
:104A9000828193810C5F1F4F06C06081718180E02D
:104AA00090E00E5F1F4FA4010E944126A82EA81877
:104AB000FB2DFF77BF2EB6FE0BC02B2D2E7FA5142E
:104AC00050F4B4FE0AC0B2FC08C02B2D2E7E05C0E7
:104AD0007A2C2B2D03C07A2C01C0752C24FF0DC01D
:104AE000FE01EA0DF11D8081803311F4297E09C099
:104AF00022FF06C07394739404C0822F867809F055
:104B0000739423FD13C020FF06C05A2C731418F4AD
:104B1000530C5718732C731468F4B70180E290E0BB
:104B20002C870E94BF2373942C85F5CF731410F447
:104B3000371801C0312C24FF12C0B70180E390E088
:104B40002C870E94BF232C8522FF17C021FF03C0A2
:104B500088E590E002C088E790E0B7010CC0822FA2
:104B6000867859F021FD02C080E201C08BE227FD6A
:104B70008DE2B70190E00E94BF23A51438F4B7017D
:104B800080E390E00E94BF235A94F7CFAA94F401E7
:104B9000EA0DF11D8081B70190E00E94BF23A110B2
:104BA000F5CF332009F451CEB70180E290E00E94A6
:104BB000BF233A94F6CFF7018681978102C08FEF29
:104BC0009FEF2C96E2E10C94C326DC01CB01FC01A3
:104BD000F999FECF06C0F2BDE1BDF89A319600B456
:104BE0000D9241505040B8F70895F999FECF92BD0B
:104BF00081BDF89A992780B50895A8E1B0E042E018
:104C000050E00C94E725DC01A40FB51F4150504043
:104C100048F0CB01840F951F2E910E94142641501D
:104C20005040D0F70895262FF999FECF92BD81BD4F
:104C3000F89A019700B4021639F01FBA20BD0FB6DA
:104C4000F894FA9AF99A0FBE08950196272F0E94B8
:104C500014260C941326FC0105906150704001103D
:104C6000D8F7809590958E0F9F1F0895FC01615095
:104C7000704001900110D8F7809590958E0F9F1F7E
:104C80000895FA01AA27283051F1203181F1E894E2
:104C90006F936E7F6E5F7F4F8F4F9F4FAF4FB1E02F
:104CA0003ED0B4E03CD0670F781F891F9A1FA11D2A
:104CB000680F791F8A1F911DA11D6A0F711D811D2B
:104CC000911DA11D20D009F468943F912AE0269FF0
:104CD00011243019305D3193DEF6CF010895462F4F
:104CE0004770405D4193B3E00FD0C9F7F6CF462F30
:104CF0004F70405D4A3318F0495D31FD4052419399
:104D000002D0A9F7EACFB4E0A69597958795779555
:104D10006795BA95C9F700976105710508959B01DC
:104D2000AC010A2E06945795479537952795BA9565
:104D3000C9F7620F731F841F951FA01D0895B7FF49
:104D40000C9451210E945121821B930B08952F92A4
:104D50003F924F925F926F927F928F929F92AF920B
:104D6000BF92CF92DF92EF92FF920F931F93CF9358
:104D7000DF93CDB7DEB7CA1BDB0B0FB6F894DEBFEF
:104D80000FBECDBF09942A88398848885F846E8415
:104D90007D848C849B84AA84B984C884DF80EE805F
:104DA000FD800C811B81AA81B981CE0FD11D0FB668
:104DB000F894DEBF0FBECDBFED010895F894FFCF8C
:104DC0003FC80000003200000096000000FEFFFF18
:104DD0000A0A0A0A6E2F02005749444532000100B0
:104DE00057494445310041505A4D444D4E4F43417F
:104DF0004C4C0101010101010000C206200001002C
:024E00000000B0
:00000001FF
